:020000000628D0
:04000C00D02882076F
:1000100080340834983410349834043480340434F0
:1000200072340434AA341034AA34043498340434B6
:100030008F3408345F3410345F340434653404344E
:100040008034043472340434803410348034043402
:100050007234043472340834723404345534023443
:100060005F340834653404345F3404347234083443
:1000700080341034BF340434AA3404349834043443
:1000800072341034803404348F340434983404349B
:10009000BF340434BF34103482075F341034553415
:1000A00004344C340834403408344034083439348F
:1000B0000834403408344C3408345F341034553438
:1000C00004344C3408344C340834553408345F3428
:1000D0000834553410345F341034553404344C34FF
:1000E0000834403408344034083439340834403457
:1000F00008344C3408345F341034553410344C34E4
:1001000008344C340834553408345F3410344834DF
:10011000083448340834393408343934083439342C
:10012000083440340834403408344C3408345F34E4
:100130000834553410345F341034553404344C349E
:1001400008344034083440340834393408344034F6
:1001500008344C3408345F341034553404344C348F
:1001600008344C34083455340834553408345F347A
:1001700020348207BF341034BF340434BF34083411
:10018000BF340434BF34083498340434AA340834F7
:10019000BF340434BF340834CA340834BF34103494
:1001A00003138316113085000F30860088308100DC
:1001B0008312850186010C3084008001840A041FAB
:1001C000DD2817081A3E9700F92010215F217E21B3
:1001D000C921013A031D312AA80A892289228922CC
:1001E0001708343A031DE6281608033A031DE628CB
:1001F0005F2A06080F39003A031908000030890009
:1002000088018316081555308900AA3089008814A2
:100210000811881809298312023093004B21080025
:100220009001A70A2708033994008922B6211030CB
:100230009300100807209100900A100807209200F0
:1002400030218601900A1008443A031990010608EB
:100250000F39003A03191129023093004B2108008D
:100260008E010E0812060319080013088D001108EC
:1002700085144021851040218D0B37298E0A3129A4
:100280008C000000000000000000000000000000E2
:100290008C0B412908009101910901309200302115
:1002A000910B4D298922892289228922892289223A
:1002B0008922892208000108033994000800851169
:1002C00005155B211708840003101608003A03196E
:1002D0007529013A03197329033A03197129940DF9
:1002E000940D940D940D940D940D00081404800049
:1002F000960A161D08009601970A080098011A3000
:100300009900190884000008A7001808003A03198A
:100310009529013A03199329033A03199129A70C46
:10032000A70CA70CA70CA70CA70C2708033994004F
:10033000AB21892289228922980A1819A82918082C
:100340001606031D812919081706031908008129BB
:100350009801990A9F29B62191002030920010300F
:10036000051E013093003021860108001408003A70
:100370000319C129013A0319C329033A0319C529ED
:10038000C72906165F3486164C3406174034861784
:1003900033340511851598011A3099001908840025
:1003A0000008A7001808003A0319E229013A0319C6
:1003B000E029033A0319DE29A70CA70CA70CA70C08
:1003C000A70CA70C270803399400FC21003A031955
:1003D000003415081406031D0034980A1819F92969
:1003E00018081606031DCE2919081706031901342B
:1003F000CE299801990AF02995010730051E03308E
:100400008E00FF308D00FF308C000618142A8618ED
:10041000182A06191C2A8619202A8C0B052A8D0BEE
:10042000032A8E0B012A0034061695015F30242A18
:10043000861615144C30242A061795144030242AA9
:100440008617151495143330910020309200033034
:100450009300302106080F39003A031D292A86012E
:100460000134013093004B21013093004B217E2158
:10047000013093004B21013093004B2189228922C6
:100480008922003089008316081483120808280284
:1004900003185F2A90011030930089221008B920B8
:1004A0009100900A1008B92092003021900A10089B
:1004B000163A031D4D2A892289228922D928003023
:1004C0008900280888008316081555308900AA304D
:1004D00089008814081188186B2A83129001A70AD2
:1004E0002708033994008922B621053093001008AB
:1004F0004C209100900A10084C2092003021860177
:10050000900A10086C3A031D6F2A892289228922D9
:10051000D928C3308D00FF308C008C0B8D2A8D0BB9
:040520008B2A08001A
:02400E00F33F7E
:00000001FF
